:1000000003C003C003C003C003C003C003C003C0D8
:1000800013C02AC029C028C027C026C025C024C04C
:1000900023C022C021C020C01FC01EC01DC01CC064
:1000A0001BC01AC019C018C00000000000000000EA
:1000B0000000000000000000000000000000000040
:1000C000000000000000000011241FBECFEFD2E0AE
:1000D000DEBFCDBFC9D3E1C3D3CF009709F40895E4
:1000E000E0EAFFE03197F1F70197F7CF807C9B01C1
:1000F000205C3F4FDB01FC01E61BF70BEA0FFB1F07
:10010000459154914D935D93A217B307A1F70895BC
:10011000FC01E07C93E090935700E89507B600FC63
:10012000FDCF0895CF93DF939B01205C3F4FDB0110
:10013000FC01E61BF70BEA0FFB1FCD91DD9141E0BF
:100140000E0140935700E8951124A217B30781F7D9
:1001500025E0FC0120935700E89507B600FCFDCF91
:10016000DF91CF910895CF93DF93CDB7DEB7C05421
:10017000D1090FB6F894DEBF0FBECDBFBE016F5FD1
:100180007F4F90E080E0B2DFFE013196CE018F5BC1
:100190009F4F2FEF3FEF21933193E817F907C9F7EE
:1001A00090E080E0B5DFBE016F5F7F4F90E080E0C0
:1001B000B9DFC05CDF4F0FB6F894DEBF0FBECDBF16
:1001C000DF91CF910895EF92FF920F931F93CF93FA
:1001D000DF93CDB7DEB7C054D1090FB6F894DEBFB8
:1001E0000FBECDBF10E000E045E00237140774F009
:1001F000C05CDF4F0FB6F894DEBF0FBECDBFDF91FE
:10020000CF911F910F91FF90EF90089530E020E083
:10021000F801EA50FD4FE20FF31FC9018E7F48E05D
:10022000E836F407ECF44591549161E070E06C0F0E
:100230007D1F860F971FFC01518340832E5F3F4F28
:100240002034310529F77801F6EEFF1AC70160DF87
:10025000BE016F5F7F4FC70165DF005C1F4FC4CFDA
:1002600041E050E04C0F5D1F840F951F4FEF5FEF93
:10027000E2CF0F931F93CF93DF93CDB7DEB7C05478
:10028000D1090FB6F894DEBF0FBECDBFFE01319687
:10029000CE018F5B9F4F8F012FEF3CEC2193319369
:1002A000E817F907C9F790E080E032DFB80190E085
:1002B00080E038DFC05CDF4F0FB6F894DEBF0FBEC2
:1002C000CDBFDF91CF911F910F910895CF9384B14E
:1002D000836084B92998CAEF81E090E0FEDE299A14
:1002E00081E090E0FADE2998C150B1F7CF910895EE
:1002F000F0E0E0E0099416C019FC400593111500E8
:10030000090212000101008032090400000000000F
:10031000000012011001FF000008D016530706026A
:100320000000000111241FBECFEFD2E0CDBFDEBF21
:1003300021E0A0E0B1E001C01D92AC32B207E1F7CC
:1003400030C1DC0180E090E041E050EA609530E0AF
:1003500009C02D9182279795879510F084279527BE
:10036000305EC8F36F5FA8F38D939D930895CF938C
:10037000DF93CC27C395499BE9F7499B0BC0499B69
:1003800009C0499B07C0499B05C0499B03C0499BC5
:1003900001C089C00F92C0910E01DD27CA5EDE4FF9
:1003A0000F9065E5499B03C00F920F90E6CF0F9326
:1003B0000F910F9320E040E10F9109B1067001FB0E
:1003C00027F93F9350E03BE039C0167040642F7727
:1003D000012F5F5F1EC0406819B116702F77525011
:1003E0001FC0406409B12F770670D1F15F5F00C074
:1003F00023C0406219B12F77167091F15F5F00C082
:1004000025C006701027515012F45D5F0000115096
:1004100027952C3F19B1C8F6167001270150279572
:100420002C3FC8F64227499309B1067010274F7335
:10043000115027952C3FA8F64695469519B1167090
:1004400079F00127015027952C3F98F66B5A60F3FD
:10045000315009B1B0F600C014E01BBB00271DC02D
:100460003B503195C31BD04014E01BBB0881033CBB
:10047000E9F00B34D9F020910C011981110F1213FE
:10048000EDCF093611F10D3211F0013E39F7CAE016
:100490001BB312FD02C0CA95D9F7009314013F9116
:1004A000CBB3C2FD67CFDF91CF91089520911401A6
:1004B0002223A9F310911201112309F534300AF116
:1004C0003093120120930D011CC0009112010130E4
:1004D000B4F40AE530910F0134FD14C000930F010C
:1004E000C1E0D1E013C0052710E000C000000BB947
:1004F0001AC0052710E0221F1DC010E021C04AE5E8
:1005000002C032ED432FC4E1D0E032E01AB11660F0
:10051000599A0BB11AB956E020E865E320FF052788
:100520000BB9279517951C3FF0F66695B8F7B1F70C
:1005300020FF05270BB9279517951C3FD0F6279567
:10054000179517FF052700001C3F0BB9B0F629913E
:100550003A9519F7097F10911301110FC651D04038
:100560000BB911F010930C0114E01BBB02601AB11F
:10057000197F402F497F54E05A95F1F70BB91AB90A
:100580004BB98DCFF201309711F48FEF9CEC21E045
:100590000C0120935700E8951124CF0102962C01FD
:1005A0000895499B03C004B600FC06C0EDEFF9E1D5
:1005B000E491EF3F09F0F1C0A89580916000886157
:1005C0008093600010926000519A88EB9BE0E0E914
:1005D000F1E03197F1F70197D1F751988AE58093CF
:1005E0000F018FEF8093000180916D0084608093F4
:1005F0006D0080916800846080936800509A34E7B1
:10060000632E34E0732E312C512C412CC5EDD4E1F6
:1006100084E699B1967009F084E6815041F4109215
:10062000130110920C0120EC622E23E0722EDA9B53
:10063000A4C09DDE84E08BBBA89522E032120CC0E2
:10064000E0E0FAE1E054F10983E080935700E89597
:100650003097C1F7512C412C832D803409F091C083
:10066000F2013297E1158AE1F80720F485E08093E2
:100670005700E895312C80911201835087FD2FC0DF
:1006800090910D019D3221F5883011F5809117016F
:1006900093EC909301019AE590930F0190911801CA
:1006A000807609F4A4C0712C91117BC082E09AE19C
:1006B000909311018093100188E090911E01911197
:1006C00005C090911D01981708F4892F80930001AF
:1006D0001092120180911701807609F0712C80919F
:1006E0000F0184FF30C0809100018F3F61F1C82F5E
:1006F000893008F0C8E0982F9C1B909300019091DE
:10070000010128E8922790930101882381F0E0916C
:100710001001F0911101A2E0B1E08C2F94919D9312
:1007200031968150D9F7F0931101E09310016C2FAD
:1007300082E091E006DECC5FCC3019F08FEF809341
:100740000001C0930F01C30101963C01803B24E0EE
:10075000920729F4EDEFF9E1E491EF3FC1F48C74D5
:1007600009F480C05898DA9B51CF8CE1499B8CE109
:100770008150E1F784E08BBB49CF219709F049CF45
:100780005BCF843009F076CFCD2B09F074CF589829
:100790001AB81092680010926D0084B78EBB14BE18
:1007A000A8CD913079F44114510411F480E085CF43
:1007B00080911B01807C482E50901C0181E187BFF5
:1007C000E895F4CF933081F48091190190911A014A
:1007D000D9DE80911B0190911C01D4DE842D8F7392
:1007E00029F790E4392E69CF9F73392EDFCF2091FE
:1007F000190110920A0191110AC010920B012AE00E
:1008000031E082E0309311012093100156CF9530F2
:1008100029F4209313012AE031E0F4CF963091F4CB
:1008200080911A01813041F48CE19AE19093110199
:100830008093100182E141CF823009F0B7CF8AE086
:100840009AE1F4CF983051F0993019F420931501C2
:10085000E2CF81E09A30F9F280E0DDCF25E131E0AE
:1008600081E0D0CF589A7FCF85B115B884B18FEF92
:1008700084B98AEF90E031DC84B114B88AEF90E05B
:100880002CDCF89470DC9FDCF4DC20DD8DEF99E14A
:0E0890003FDC2EDD90E080E00895F894FFCF6D
:040000030000008079
:00000001FF
